:100000000C94F0030C9434040C9434040C943404D5
:100010000C9434040C9434040C9434040C94340480
:100020000C9434040C9434040C94210E0C94F30EB0
:100030000C9434040C9434040C9434040C94340460
:100040000C9434040C9478230C9434040C943404ED
:100050000C9434040C94091D0C9434040C94340452
:100060000C9434040C9434040C9434040C94340430
:100070000C9434040C9434040C9434040C94340420
:100080000C9434040C9434040C9434040C94340410
:100090000C9434040C9434040C9434040C94340400
:1000A0000C9434040C9434040C94340444044E042E
:1000B00066047E04C604CC04ED04D204E804DE0425
:1000C000E304D804AE049604F204600F820F7010AB
:1000D000820F7010C70FEA0F70103F1052103413C8
:1000E000341363136313A613E413FD15FD15FD13F9
:1000F000FD15FE14FE14D115FD15FD15E81501E1E1
:100100000137023702E10138023801E201250225F8
:1001100002E20001E10137023702E1013802380151
:10012000E10130023002E10001E10137023702E172
:100130000138023801E10107020702E1000135023E
:1001400035012002200001E10137023702E10138C8
:10015000023801E10125022502E10001E101360238
:100160003602E10138023801E10125022502E100F1
:1001700001E10136023602E10138023801E10126CF
:10018000022602E10001E10137023702E1013802F3
:100190003801E10126022602E10002E002E201301C
:1001A00002300002E002E20001E001E20002E002AF
:1001B000E3016402640002E002E30001E001E30005
:1001C00002E002E2012E022E02E10002E002E10260
:1001D000E20001E001E101E20002E001E3010602C8
:1001E0000602E30002E00001E00002E001E3011981
:1001F000021902E30002E00001E0000000F0A1F0BB
:10020000A329002B00E200E100358100001E00144C
:100210000004001D710D304D831F001A0016001BD5
:10022000000C304C00200008000700060052002A95
:1002300000210015000900190051004A0022001792
:10024000000A00050000000330E101E3000000E2C5
:1002500000000002543100E7000000E60000000446
:100260005423001C000B00110000002E7F240018F6
:10027000000D00100050004B0025000C000E003651
:10028000004F002C00260012000F003700E1082864
:10029000002700130033003871E1044E002D002FB9
:1002A000003474E50030810000010001000100010C
:1002B00000010000003A003500310001000100019A
:1002C000003B0035022102350001004C003C001EBD
:1002D0000224062202010001003D002D0224022416
:1002E00004010001003E000100370011040000017C
:1002F000000100010000000100000001000E3001BB
:100300000000000100000068003F002406240224D1
:100310000400004500400022042502110431026956
:100320000041002304260264005000010042003511
:100330000025045200510001004300350226043814
:10034000004F006A0044001E02310021020100003B
:100350000001000100010001000100000001000196
:100360000001000100010001000100F400F200FBA7
:1003700000010001000100F000F100FA000100019D
:10038000000100F500F300FC00010001000100F98C
:1003900000FA00F600000001000100010000000169
:1003A0000000000100A800010000000100000001A1
:1003B0000001000100A900AA0000000100010001E5
:1003C000000100010001000100010001000100AC7A
:1003D000000100B600010001000100AB0050000167
:1003E00000010001000100520051000100AE0001B7
:1003F00000010001004F00000001000100010001A8
:1004000000010000000100010001000100010001E5
:1004100000010001000100010001000100010001D4
:1004200000010001000100010001000100010001C4
:1004300000010001000100010001000100000001B5
:100440000001000100000001000000010004300173
:1004500000000001000000010005300630093001F5
:1004600000000001000A300B3008300100010001DB
:10047000000100073001000100010001000100013E
:100480000001000100010001000100010001000164
:100490000001000100010001000100010001000055
:1004A0000001000100010001000100000001000145
:1004B00000010001000100010001000100500001E5
:1004C0000001000100010052005100010001000183
:1004D00000010001004F00010001000100010001C6
:1004E0000001000100000001000100010000000106
:1004F00000000001000100010000000100000001F7
:10050000003F00520051002302000001004000247F
:100510000021001E00270001004100250022001FCD
:1005200000370001004200260023002000360001B1
:10053000004300300230002402270201004400453D
:1005400000380001000100000001000100E100018D
:1005500000E0000000010001000100010001003D79
:100560000001000100010001000100E000010001A4
:10057000000100010001002C000100010001000148
:100580000001003C00010001000100010000003AF0
:1005900000010001000000010000003B000E3001DE
:1005A0000000000100000001000100010001000145
:1005B0000000000100010001000100010001000134
:1005C0000001000100010001000100010001000123
:1005D0000001000100010001000100010001000113
:1005E0000001000100010001000100010001000004
:1005F0000016034500720067006F0044006F00782A
:1006000000200045005A00000016034500720067F4
:10061000006F0044006F007800200045005A000081
:10062000000403090409026D00040100A0FA090492
:1006300000000103010100092111010001223F0016
:100640000705810308000A090401000103010200F3
:10065000092111010001224D000705820308000A4B
:100660000904020001030000000921110100012218
:1006700036000705830308000A090403000103008C
:10068000000009211101000122390007058403102F
:1006900000011201100100000008EDFE0713010027
:1006A0000102000105010906A101050719E029E77A
:1006B0001500250195087501810205081901290514
:1006C00095057501910295017503910105071900C2
:1006D000297715002501957875018102C00501096A
:1006E00080A101850216010026B7001A01002AB771
:1006F00000751095018100C0050C0901A101850359
:10070000160100269C021A01002A9C027510950110
:100710008100C005010902A1010901A10005091913
:1007200001290515002501950575018102950175C1
:100730000381010501093009311581257F95027575
:1007400008810609381581257F9501750881060500
:100750000C0A38021581257F950175088106C0C0F5
:1007600005010906A101050719E029E71500250182
:100770009508750181029501750881010508190127
:1007800029059505750191029501750391010507EC
:10079000190029FF150025FF950675088100C00086
:1007A00000000000000000000000010204060A0F23
:1007B00017202C3A4A5D71879DB3C7DAE9F5FCFF33
:1007C000FCF5E9DAC7B39D87715D4A3A2C20170F13
:1007D0000A06040201000000000000000000000002
:1007E00011241FBECFEFDAE0DEBFCDBF04B603FE9B
:1007F00024C08091F0019091F101A091F201B0919B
:10080000F3018730904BA740B04BB9F41092F00140
:100810001092F1011092F2011092F30114BE84B70C
:10082000877F84BF88E10FB6F894809360001092B0
:1008300060000FBEE0E0FFE3099511E0A0E0B1E049
:10084000E4E7FAE402C005900D92A433B107D9F7AA
:1008500011E0A4E3B1E001C01D92A03FB107E1F7B0
:100860000E94650B0C9438250C940000462F50E034
:100870004F30510508F0DEC0DC01FA01EA5AFF4FA3
:1008800012968C910C94ED24882321F085EE0E9421
:10089000D111D0C085EE0E949912CCC0882349F0B6
:1008A0000E94D31C909335018093340188EF91E02E
:1008B000089580913401909135010E94DF1C8739A1
:1008C00091050CF0A8C08AEE91E00895882349F0C4
:1008D0000E94D31C909335018093340187EE91E000
:1008E000089580913401909135010E94DF1C873971
:1008F00091050CF093C089ED91E00895882349F0AB
:100900000E94D31C909335018093340182ED91E0D5
:10091000089580913401909135010E94DF1C873940
:1009200091050CF07EC080EC91E00895882349F099
:100930000E94D31C90933501809334018BEB91E09E
:10094000089580913401909135010E94DF1C873910
:1009500091050CF069C08DEA91E00895882349F073
:100960000E94D31C909335018093340188EA91E072
:10097000089580913401909135010E94DF1C8739E0
:1009800091050CF054C08AE991E00895882309F498
:1009900051C085E891E00895882309F44BC080E7B1
:1009A00091E00895882309F445C08BE591E008950E
:1009B000882309F43FC086E491E008958823D1F1AB
:1009C0008DE391E008958823A9F188E291E00895EC
:1009D000882381F183E191E00895882359F18EEF16
:1009E00090E00895882331F18091B3019091B40192
:1009F000A091B501B091B60120E2822780729927BB
:100A0000AA27BB278093B3019093B401A093B501AB
:100A1000B093B6010FC085EF91E0089584EE91E0A8
:100A200008958BEC91E0089586EB91E0089583EAB8
:100A300091E0089580E090E0089508956091B301F9
:100A40007091B4018091B5019091B6010E94381C5B
:100A500056985E9825982D9826982E9827982F9826
:100A60008330C1F028F4813041F0823049F008959C
:100A7000843049F0853051F00895259A2D9A0895D3
:100A8000269A2E9A0895259A2D9A04C0259A2D9A71
:100A9000269A2E9A279A2F9A08950C941E055698F6
:100AA0005E9825982D9826982E9827982F988FEF46
:100AB00090E0909389008093880090938B008093BE
:100AC0008A0090938D0080938C00259A2D9A2FEFA9
:100AD00080E792E0215080409040E1F700C00000A4
:100AE000269A2E9A2FEF80E792E021508040904086
:100AF000E1F700C00000279A2F9A2FEF80E792E0DD
:100B0000215080409040E1F700C0000025982D98CA
:100B10002FEF80E792E0215080409040E1F700C045
:100B2000000026982E982FEF80E792E02150804019
:100B30009040E1F700C0000027982F9856985E98E3
:100B400025982D9826982E9827982F98089589EA09
:100B50008093800089E08093810024982C983F98AE
:100B60008AB18F748AB96E98479A8BB1806B8BB9B2
:100B7000769A0E944F050C941D0580E28093000137
:100B80008091360181110EC00E940C0681E0809395
:100B900036012FEF83ED90E3215080409040E1F744
:100BA00000C0000080E40E941206809300018111C1
:100BB0002EC00E943C0680930001811128C00E9433
:100BC0003C0680930001811122C08FE30E943C0605
:100BD0008093000181111BC00E94340680E40E94B2
:100BE000120680930001811112C08CE00E943C0625
:100BF0008093000181110BC00E943C06809300018C
:100C0000811105C08FE30E943C06809300010E9481
:100C100034068091000108951092B9008AE0809313
:100C2000B800089594EA9093BC009091BC0097FF9F
:100C3000FCCF9091B900987F983021F0903111F05D
:100C400081E008958093BB0084E88093BC0080918C
:100C5000BC0087FFFCCF8091B900887F883111F0FC
:100C6000803471F780E0089584E98093BC0080911E
:100C7000BC0084FDFCCF08958093BB0084E8809382
:100C8000BC008091BC0087FFFCCF9091B900987F99
:100C900081E0983209F480E0089584E88093BC00F4
:100CA0008091BC0087FFFCCF8091BB0008958091AC
:100CB0000001811115C080E40E941206809300019A
:100CC00081110CC082E10E943C06809300018111D9
:100CD00005C08FEF0E943C06809300010E943406FD
:100CE00084B1807F84B985B1807F85B98AB1837FE3
:100CF0008AB98BB1837F8BB93E98469808950E943C
:100D0000BD05809300010E94570680B38C7080BBA4
:100D100081B3836F81BBA8E3B1E0E6E4F1E08EE04C
:100D20008E0F11921D928E13FCCF0C94A705BF92CB
:100D3000CF92DF92EF92FF920F931F93CF93DF93A7
:100D400080910001882379F0809137018F5F809333
:100D50003701811108C00E94BD05809300018111F7
:100D600002C00E944F0508E311E0C0E0D0E0DD249E
:100D7000D39482E0C82EEE24E394F12CC730D10541
:100D800000F580910001811164C080E40E94120688
:100D900080930001811112C082E10E943C06809381
:100DA000000181110BC0C7010C2E01C0880F0A94ED
:100DB000EAF780950E943C06809300010E94340669
:100DC00048C0CA30A1F028F4C83059F0C93061F0E9
:100DD00005C0CC3089F070F0CD3089F0209A289889
:100DE00010C0219A29980DC0229A2A980AC0239AE5
:100DF0002B9807C0529A01C0539A5B9802C03E9A42
:100E0000469890EA9A95F1F79FB1799902C082E0ED
:100E100001C080E091709D25982B7C9902C084E0F0
:100E200001C080E0892B7D9902C038E001C030E02C
:100E3000832B7E9902C020E101C020E0822B9FB16C
:100E40009095991F9927991F9295990F907E892BBC
:100E50000FC080910001811149C080E40E941206F8
:100E600080930001882379F1B12C0E9434068B2DE8
:100E7000F8019081981719F08083C09201010E94B7
:100E8000570621960F5F1F4FCE30D10509F076CF60
:100E900080910101882361F18150809301018823B1
:100EA00039F08FE99FE00197F1F700C0000020C002
:100EB000A6E4B1E0E8E3F1E0CF01825F91919D9378
:100EC0008E13FCCF15C083E10E943C068093000185
:100ED0008111CACF81E40E94120680930001811122
:100EE000C3CF0E944D06B82EB094BFCF80E0C0CFD4
:100EF0000E944D0581E0DF91CF911F910F91FF90EE
:100F0000EF90DF90CF90BF900895E82FF0E0EA5B7C
:100F1000FE4F8081089508958B3B910578F4883ABF
:100F2000910540F5853A9105D0F48430910508F09B
:100F3000B1C08130910509F4ADC06BC0803E910510
:100F400008F467C0883E910508F4A4C09C01205FA6
:100F500031092031310508F05CC090650895853A6B
:100F6000910509F459C0863A910509F058C082E804
:100F700090E40895883A910509F454C0893A91059E
:100F800009F453C08A3A910509F452C08B3A91058D
:100F900009F451C08C3A910509F450C08D3A91057D
:100FA00009F44FC0803B910509F44EC08E3A91057B
:100FB00009F44DC08F3A910509F44CC0813B91056D
:100FC00009F44BC0823B910509F44AC0833B91056B
:100FD00009F449C0843B910509F448C0853B91055B
:100FE00009F447C0863B910509F446C0873B91054B
:100FF00009F445C0883B910509F444C0893B91053B
:1010000009F443C08A3B910509F442C080E094E4AE
:10101000089580E090E0089581E890E4089583E8E1
:1010200090E4089582EE94E4089589EE94E408959E
:101030008AEE94E4089585EB94E4089586EB94E4B5
:10104000089587EB94E408958CEC94E408958DEC76
:1010500094E4089583E895E408958AE895E4089572
:1010600082E995E4089584E995E4089581E296E49F
:10107000089583E296E4089584E296E4089585E273
:1010800096E4089586E296E4089587E296E408954A
:101090008AE296E40895089596E0799FF00111247C
:1010A00094E5899FE00DF11D1124E60FF11DEE0F6F
:1010B000FF1FEF5FFD4F859194910895880F991F51
:1010C000FC01E558FF4F859194910895880F991F71
:1010D000FC01E550FE4F85919491089526E0729FA2
:1010E000F001112444E5849FE00DF11D1124E60F69
:1010F000F11DEE0FFF1FEF5FFD4F859194919C0155
:101100003A9521154FE1340708F41AC13F512115D2
:10111000304120F49F700E94660808959C0130536E
:101120002115304118F49927906C0895811520E518
:10113000920769F40E941F164FEF84E39CE0415030
:1011400080409040E1F700C000000C942E1D8130DB
:1011500020E5920731F48091CE0181608093CE0129
:1011600008959C0130552115304108F051C0292FB8
:1011700033272F70332721303105D9F4AC01437068
:10118000552702C0220F331F4A95E2F73C68AC0195
:1011900064E0440F551F6A95E1F744275370242BF0
:1011A000352B73E0880F991F7A95E1F780769927A0
:1011B0001DC02230310529F4982F8827816F906A4D
:1011C000089523303105A9F4AC014370552721E07F
:1011D00030E002C0220F331F4A95E2F73C6843E03B
:1011E000880F991F4A95E1F7807E9770822B932B89
:1011F000089524303105E1F4AC014370552721E016
:1012000030E002C0220F331F4A95E2F73A68E7CF79
:101210009C0130572115304118F49F709062089559
:101220009C0130582115304118F49F70906A089540
:10123000803E9105E0F4803C910558F5813391059D
:1012400009F46FC048F48932910509F463C08A3209
:10125000910509F46DC072C089339105E9F08238B7
:101260009105D1F08533910509F44DC067C0833EE7
:10127000910581F138F4803E9105B9F0823E9105E7
:10128000D9F05CC0863E910561F1873E9105A1F1E0
:1012900055C00E945E0808952091E10120FD02C022
:1012A00021FF4CC080EE90E049C08091E10180FFB9
:1012B000F9CF89E390E042C08091E10182FF0EC046
:1012C0008091E10184FF03C080E090E037C083EEAD
:1012D00090E034C08091E10182FFF2CF82EE90E095
:1012E0002DC08091E10183FF0BC08091E10184FD5D
:1012F000EBCF87EE90E022C08091E10183FFF5CF34
:1013000086EE90E01BC08091E10185FF07C089E275
:1013100090E014C08091E10185FFF9CF85E390E072
:101320000DC08091E10186FF07C08AE290E006C00F
:101330008091E10186FFF9CF81E390E00E948C0764
:10134000089508950C94A109809164010895CF93A4
:10135000DF9300D01F92CDB7DEB79C018091E701EB
:10136000843019F593E099833B832A839093E900B5
:101370008FEF9091E800815095FD06C095ED9A950C
:10138000F1F700008111F5CF8091E80085FF0DC0D5
:1013900040E050E063E070E0CE0101960E94110C45
:1013A0008091E8008E778093E8000F900F900F9067
:1013B000DF91CF910895CF93DF9300D01F92CDB7E7
:1013C000DEB72091E701243021F522E029839B83B9
:1013D0008A8383E08093E9008FEF9091E800815049
:1013E00095FD06C095ED9A95F1F700008111F5CFB6
:1013F0008091E80085FF0DC040E050E063E070E0C0
:10140000CE0101960E94110C8091E8008E778093A6
:10141000E8000F900F900F90DF91CF9108952091E9
:10142000E7012430F1F422E02093E9002FEF30911E
:10143000E800215035FD06C035ED3A95F1F7000082
:101440002111F5CF2091E80025FF0BC040E050E0CE
:1014500065E070E00E94110C8091E8008E77809327
:10146000E8000895CF93DF93EC019091E701943069
:1014700009F046C080910C018823D9F080910D01BC
:101480008823B9F09093E9008FEF9091E8008150A4
:1014900095FD06C095E19A95F1F700008111F5CF11
:1014A0008091E80085FF2CC040E050E060E170E0F2
:1014B00017C081E08093E9008FEF9091E8008150A0
:1014C00095FD06C095ED9A95F1F700008111F5CFD5
:1014D0008091E80085FF14C040E050E068E070E0D3
:1014E000CE010E94110C8091E8008E778093E80075
:1014F00080E1FE01A4E5B1E001900D928A95E1F74B
:10150000DF91CF9108958091E601811109C00E9479
:10151000A60D0E94030E8091E20084608093E20099
:1015200008951092E601089508950C9465230E9491
:10153000C41C0E946B230E94A9100C94A20942E0D3
:1015400061EC81E00E94200D42E061EC82E00E94AB
:10155000200D42E061EC83E00E94200D42E161EC4D
:1015600084E00C94200D8091E901833009F455C08A
:1015700030F4813071F0823009F48EC008958A30E1
:1015800009F47AC08B3009F460C0893009F09CC03E
:1015900020C08091E801813A09F096C08091E8006E
:1015A000877F8093E8008091EC019091ED01892B79
:1015B00021F460E184E591E003C060E080E090E028
:1015C00070E00E945C0C8091E8008B778093E800CB
:1015D00008958091E801813209F076C08091EC0194
:1015E0009091ED01009719F0039709F06DC080917B
:1015F000E800877F8093E8008091E80082FD05C0C5
:101600008091E7018111F8CF5FC08091F100809354
:1016100064018091E8008B7753C08091E801813AA2
:1016200009F052C08091EC019091ED01892B09F0F5
:101630004BC08091E800877F8093E8008091E800AC
:1016400080FFFCCF80910C0136C08091E80181328F
:10165000D9F58091EC019091ED01892BA9F580914C
:10166000E800877F8093E8000E94550D8091EA0191
:1016700080930C010C941F168091E801813221F5B2
:101680008091E800877F8093E8000E94550D80914B
:10169000EB018093650108958091E801813AA1F4FE
:1016A0008091E800877F8093E8008091E80080FFC8
:1016B000FCCF809165018093F1008091E8008E77E6
:1016C0008093E8000C94550D089584B7877F84BFFC
:1016D00088E10FB6F89480936000109260000FBE0E
:1016E00090E080E80FB6F8948093610090936100D9
:1016F0000FBE0E94F8100E94A60D0E94030E80915A
:10170000E20084608093E20078940E9489100E9435
:10171000FA1082E091E00E94A4100E94532380916D
:10172000E701853069F40E94881C8091E5018823D7
:10173000B1F30E94B01C882391F30E94FB0BEFCF02
:101740000E940011ECCF292F332723303105C9F037
:1017500064F42130310581F02230310509F043C0B5
:101760008DE690E025E236E042C021323105F1F00D
:101770002232310541F137C082E190E022E936E0C2
:1017800036C099278130910541F08230910541F0B2
:10179000892B49F5E1E2F6E005C0E9E0F6E002C098
:1017A000E1EFF5E0849190E09F0121C06430D8F42E
:1017B000E62FF0E0EE0FFF1FEE5DFE4F208131813E
:1017C00089E090E014C0643070F470E0FB01EE0F2B
:1017D000FF1FE65EFE4F20813181FB01EA5EFE4F76
:1017E000808190E004C080E090E020E030E0FA01E9
:1017F00031832083089580E189BD82E189BD09B4E8
:1018000000FEFDCF8091D8008F7D8093D80080911D
:10181000E00082608093E0008091E00081FDFCCFD9
:101820000895CF92DF92EF92FF920F931F93CF9381
:10183000DF93EC018B016A010E94740D811133C0AA
:10184000C114D10439F0F60180819181081B190B74
:10185000C80FD91FE12CF12C0115110519F1809148
:10186000E80085FD16C08091E8008E778093E8003F
:10187000C114D10449F0F60180819181E80EF91E6E
:10188000F182E08285E00FC00E94740D882321F36D
:101890000AC089918093F10001501109FFEFEF1AFE
:1018A000FF0ADACF80E0DF91CF911F910F91FF9077
:1018B000EF90DF90CF9008952091EE013091EF01ED
:1018C0002617370748F06115710539F42091E800B3
:1018D0002E772093E80001C0B90140E06115710541
:1018E000A9F12091E701222309F443C0253009F42E
:1018F00042C02091E80023FD40C02091E80022FD75
:1019000032C02091E80020FFE9CF4091F300209100
:10191000F20030E0342BFC01CF016115710559F064
:101920002830310540F481918093F10061507109B4
:101930002F5F3F4FF1CF41E02830310509F040E003
:101940002091E8002E772093E800C8CF4111C9CF3D
:101950000AC08091E701882361F0853061F08091B1
:10196000E80083FD0AC08091E80082FFF2CF80E0AA
:10197000089582E0089583E0089581E0089520911C
:10198000EE013091EF012617370748F06115710518
:1019900039F42091E8002E772093E80001C0B901C6
:1019A000FC0120E06115710591F18091E701882328
:1019B00009F440C0853009F43FC08091E80083FD00
:1019C0003DC08091E80082FD2FC08091E80080FF3B
:1019D000E9CF2091F3008091F20090E0922B611505
:1019E000710559F08830910540F424912093F1005D
:1019F0003196615071090196F2CF21E0089709F004
:101A000020E08091E8008E778093E800CBCF211111
:101A1000CCCF0AC08091E701882361F0853061F066
:101A20008091E80083FD0AC08091E80082FFF2CF38
:101A300080E0089582E0089583E0089581E00895AC
:101A4000982F973058F59093E900981739F07091D6
:101A5000EC002091ED005091F00003C0242F762F70
:101A600050E021FF19C03091EB003E7F3093EB0036
:101A70003091ED003D7F3093ED003091EB0031600F
:101A80003093EB007093EC002093ED005093F00046
:101A90002091EE0027FF07C09F5FD3CF8F70809308
:101AA000E90081E0089580E008958091E80187FFD2
:101AB00011C08091E80082FD05C08091E70181118D
:101AC000F8CF11C08091E8008B770BC08091E701BF
:101AD000882349F08091E80080FFF8CF8091E800EA
:101AE0008E778093E80008952091E4003091E5001E
:101AF00095E64091EC00842F817040FF22C08091D8
:101B0000E80080FD1CC08091E701882391F08530BA
:101B100091F08091EB0085FD10C04091E400509160
:101B2000E5004217530729F39A01915011F784E019
:101B3000089582E0089583E0089581E0089580E0AB
:101B400008954091E80042FFDECF08950E94140EF0
:101B50000E941C0EE0EEF0E0808181608083E8ED61
:101B6000F0E080818F77808319BCA7EDB0E08C9185
:101B70008E7F8C9380818F7E80831092E601089502
:101B80000F931F93CF93DF930E94140E0E941C0E9D
:101B9000C8EDD0E088818F778883888180688883CA
:101BA00088818F7D888319BC1092E7011092E30130
:101BB0001092E5011092E40100EE10E0F80180813E
:101BC0008B7F808388818160888342E060E080E051
:101BD0000E94200DE1EEF0E080818E7F8083E2EEB6
:101BE000F0E0808181608083808188608083F8015B
:101BF00080818E7F8083888180618883DF91CF910F
:101C00001F910F910895E8EDF0E080818F7E808331
:101C1000E7EDF0E080818160808384E082BF81E035
:101C20008093E6010C94C00DE8EDF0E080818E7F9A
:101C300080831092E20008951092DA001092E10081
:101C400008951F920F920FB60F9211242F933F9376
:101C50004F935F936F937F938F939F93AF93BF93B4
:101C6000EF93FF938091E10082FF0BC08091E2002F
:101C700082FF07C08091E1008B7F8093E1000E948A
:101C800088108091DA0080FF1FC08091D80080FF0B
:101C90001BC08091DA008E7F8093DA008091D9009A
:101CA00080FF0DC080E189BD82E189BD09B400FEDD
:101CB000FDCF81E08093E7010E94830A05C019BC33
:101CC0001092E7010E94910A8091E10080FF19C003
:101CD0008091E20080FF15C08091E2008E7F8093AA
:101CE000E2008091E20080618093E2008091D80060
:101CF00080628093D80019BC85E08093E7010E9440
:101D0000950A8091E10084FF30C08091E20084FF59
:101D10002CC080E189BD82E189BD09B400FEFDCF00
:101D20008091D8008F7D8093D8008091E1008F7ED4
:101D30008093E1008091E2008F7E8093E2008091A9
:101D4000E20081608093E2008091E301882311F03A
:101D500084E007C08091E30087FD02C081E001C0FC
:101D600083E08093E7010E94970A8091E10083FF5E
:101D700029C08091E20083FF25C08091E100877F28
:101D80008093E10082E08093E7011092E30180916B
:101D9000E1008E7F8093E1008091E2008E7F80934E
:101DA000E2008091E20080618093E20042E060E026
:101DB00080E00E94200D8091F00088608093F00008
:101DC0000E94940AFF91EF91BF91AF919F918F91E3
:101DD0007F916F915F914F913F912F910F900FBE27
:101DE0000F901F9018951F920F920FB60F9211240B
:101DF0002F933F934F935F936F937F938F939F9313
:101E0000AF93BF93CF93DF93EF93FF93C091E9001C
:101E1000CF708091EC00D82FD17080FDD0E8109267
:101E2000E9008091F000877F8093F00078940E9411
:101E3000370F1092E9008091F00088608093F000E5
:101E4000CD2BCF70C093E900FF91EF91DF91CF913F
:101E5000BF91AF919F918F917F916F915F914F91C2
:101E60003F912F910F900FBE0F901F9018951F93C9
:101E7000CF93DF93CDB7DEB7AA970FB6F894DEBF46
:101E80000FBECDBFE8EEF1E088E08E0F9091F1003B
:101E900091938E13FBCF0E94B30A8091E80083FFD9
:101EA0001FC18091E8019091E901492F50E04A302B
:101EB000510508F015C1FA01EB59FF4F0C94ED24C0
:101EC000803881F0823809F00BC18091EC018F706D
:101ED0008093E9008091EB0085FB882780F91092C0
:101EE000E90006C08091E4019091E50191118260C2
:101EF0009091E800977F9093E8008093F100109212
:101F0000F100C8C0282F2D7F09F0EAC0882319F0FE
:101F1000823061F0E5C08091EA01813009F0E0C0D3
:101F2000933009F080E08093E5012BC08091EA01B5
:101F3000811127C08091EC018F7009F4D1C080938A
:101F4000E9002091EB0020FF1CC0933021F4809128
:101F5000EB00806214C09091EB0090619093EB00D5
:101F600021E030E0A90102C0440F551F8A95E2F735
:101F70004093EA001092EA008091EB008860809321
:101F8000EB001092E9008091E800877F86C0811104
:101F9000A7C01091EA011F778091E3008078812B20
:101FA0008093E3008091E800877F8093E8000E949F
:101FB000550D8091E80080FFFCCF8091E3008068A0
:101FC0008093E300111102C082E001C083E080939E
:101FD000E70186C08058823008F082C08091EA0113
:101FE0009091EB018C3D53E0950779F583E08A836E
:101FF0008AE289834FB7F894DE01139620E03EE031
:1020000051E2E32FF0E050935700E49120FF03C02A
:10201000E295EF703F5FEF708E2F90E0EA3010F0A6
:10202000C79601C0C0968D939D932F5F243149F7C9
:102030004FBF8091E800877F8093E8006AE270E0FC
:10204000CE0101960E945C0C14C0AE014F5F5F4F41
:102050006091EC010E94A30BBC01892B09F440C0E4
:102060009091E800977F9093E80089819A810E947F
:10207000BF0C8091E8008B778093E80031C08038F6
:1020800079F58091E800877F8093E8008091E301F3
:102090008093F1008091E8008E778093E8000E94A1
:1020A000550D1EC081111CC09091EA019230C0F400
:1020B0008091E800877F8093E8009093E3010E947D
:1020C000550D8091E301811106C08091E30087FDE9
:1020D00002C081E001C084E08093E7010E949F0A72
:1020E0008091E80083FF0AC08091E800877F809399
:1020F000E8008091EB0080628093EB00AA960FB617
:10210000F894DEBF0FBECDBFDF91CF911F91089530
:102110000895CF938091E7018823A1F0C091E90051
:10212000CF709091EC00892F817090FD80E8C82BD2
:102130001092E9008091E80083FD0E94370FCF7074
:10214000C093E900CF91089590936B0180936A0149
:102150000895E0916A01F0916B01309721F00190B0
:10216000F081E02D099480E00895E0916A01F091FA
:102170006B01309721F00280F381E02D09940895DE
:10218000E0916A01F0916B01309721F00480F581B4
:10219000E02D09940895209168013091690182171A
:1021A000930771F09093690180936801E0916A014F
:1021B000F0916B01309721F00680F781E02D0994B2
:1021C000089520916601309167018217930771F09D
:1021D0009093670180936601E0916A01F0916B0131
:1021E000309721F00084F185E02D09940895089539
:1021F0000C94F7100E94CA1C0E947F060C94901D3C
:10220000CF92DF92EF92FF920F931F93CF93DF93C2
:10221000CDB7DEB72B970FB6F894DEBF0FBECDBF9C
:102220000E9497068DE6C82E81E0D82E00E010E0CF
:10223000E02E802F0E948507F60141916F01F42E58
:10224000F826B1F40F5F1F4F0E30110589F78FEF9D
:1022500089838A831B820E94D31C8160782F9D838F
:102260008C8349815A816B818D810E94A31140C06A
:102270009091CE0191FF04C08B870E948B078B85C4
:1022800020E030E04F2D50E0922FBA01022E02C024
:10229000759567950A94E2F760FF24C02E83EF825C
:1022A00021E030E0690102C0CC0CDD1C9A95E2F718
:1022B00090E08C219D21892B09F420E028870E9441
:1022C000D31C8160782F9A8789874E815F816885CA
:1022D0008A850E94A311F801E359FE4F8081C82628
:1022E000C08206C02F5F3F4F2630310569F6AACF66
:1022F0000E94772010916C010E94A9101817A1F07C
:102300000E94A91080936C012B960FB6F894DEBF43
:102310000FBECDBFDF91CF911F910F91FF90EF9036
:10232000DF90CF900C94A2092B960FB6F894DEBFE5
:102330000FBECDBFDF91CF911F910F91FF90EF9016
:10234000DF90CF900895CF93DF93CDB7DEB72B9773
:102350000FB6F894DEBF0FBECDBF4F835887698795
:102360007A878B87DE01119686E0FD0111928A95AE
:10237000E9F785E0FE01379601900D928A95E1F725
:1023800049815A816B817C818D819E810E94B9181F
:102390002B960FB6F894DEBF0FBECDBFDF91CF9165
:1023A0000895CF93882309F4C2C0C82F823859F406
:1023B0000E94A91081FDBBC089E30E94551B0E94A9
:1023C000121C89E30CC0833879F40E94A91080FDA7
:1023D000AEC083E50E94551B0E94121C83E50E943B
:1023E000971BCF910C94121C843859F40E94A910A9
:1023F00082FD9DC087E40E94551B0E94121C87E449
:10240000EECF8CEF8C0F813A48F48C2F0E94B822CB
:1024100081118DC08C2F0E94551BE3CF80E28C0F61
:10242000883048F4C77081E001C0880FCA95EAF788
:102430000E94DB1BD6CF8BE58C0F833078F4C53A36
:1024400029F0C63A31F083E890E005C081E890E0D9
:1024500002C082E890E0CF910C94CB1088E58C0FFD
:10246000833108F064C0C83A39F1C93A41F1CA3A37
:1024700049F1CB3A51F1CC3A59F1CD3A61F1C03B37
:1024800069F1CE3A71F1CF3A79F1C13B81F1C23BAA
:1024900089F1C33B91F1C43B99F1C53BA1F1C63B26
:1024A000A9F1C73BB1F1C83BB9F1C93BC1F1CA3B86
:1024B000C9F180E090E038C082EE90E035C089EE4E
:1024C00090E032C08AEE90E02FC085EB90E02CC007
:1024D00086EB90E029C087EB90E026C08CEC90E082
:1024E00023C08DEC90E020C083E891E01DC08AE815
:1024F00091E01AC082E991E017C084E991E014C02C
:1025000081E292E011C083E292E00EC084E292E0A8
:102510000BC085E292E008C086E292E005C087E247
:1025200092E002C08AE292E0CF910C94E110CF9148
:102530000895882309F44BC0823859F40E94A910E9
:1025400081FF45C089E30E94551B0E94121C89E34C
:102550000CC0833871F40E94A91080FF38C083E555
:102560000E94551B0E94121C83E50E94971B0C942D
:10257000121C843859F40E94A91082FF28C087E4F5
:102580000E94551B0E94121C87E4EFCF9CEF980F0E
:10259000913A58F390E2980F983050F4877091E098
:1025A00001C0990F8A95EAF7892F0E94E11BDFCFBE
:1025B0009BE5980F933020F480E090E00C94CB10D2
:1025C000885A833120F480E090E00C94E110089563
:1025D000882321F00E94DB1B0C94121C0895882391
:1025E00021F00E94E11B0C94121C0895BF92CF921F
:1025F000DF92EF92FF920F931F93CF93DF9300D060
:1026000000D000D0CDB7DEB725E0FC01DE01119689
:1026100001900D922A95E1F7FC0140813181028100
:10262000258122952F7063817481672B09F4E5C29F
:102630003F3F19F44F3F09F4E0C27C0149833A83DC
:1026400089819A812E830E94141B182FB92E0E9413
:10265000131B0E94DA19EB2DE295EF70F0E0E159BF
:10266000FF4F2E810C94ED248B2D807F9B2D9F702E
:10267000F92E882319F0F29480EFF822002349F014
:10268000FF2009F467C28F2D0E94EB1B0E94121CD1
:1026900061C2812F0E949912FF2009F4AEC28F2DD2
:1026A0000E94F11B26960FB6F894DEBF0FBECDBF79
:1026B000DF91CF911F910F91FF90EF90DF90CF901E
:1026C000BF900C94121C3B2D307F8B2D8F703032BD
:1026D00011F08295807F112319F0113021F12CC067
:1026E0000023B9F0222309F4A0C1213009F09DC1D3
:1026F00026960FB6F894DEBF0FBECDBFDF91CF9107
:102700001F910F91FF90EF90DF90CF90BF900C94AE
:10271000FB1B222319F0213009F46FC28E830E9423
:10272000FE1B8E8196C1002321F0223008F065C285
:102730007CC1211162C28DC1002321F0222309F442
:1027400074C108C2222309F484C119C22B2D269515
:102750002695237030E02115310521F02130310517
:10276000D1F04BC2002321F0812F9B2D937002C02A
:1027700080E090E026960FB6F894DEBF0FBECDBF86
:10278000DF91CF911F910F91FF90EF90DF90CF904D
:10279000BF900C94CB10002321F0812F9B2D9370C0
:1027A00002C080E090E026960FB6F894DEBF0FBE20
:1027B000CDBFDF91CF911F910F91FF90EF90DF90F0
:1027C000CF90BF900C94E110812F002319F00E944C
:1027D0007F1F02C00E94E71F26960FB6F894DEBF47
:1027E0000FBECDBFDF91CF911F910F91FF90EF9062
:1027F000DF90CF90BF900C946C208B2D837009F0EC
:102800007BC00111FAC1812F829586958770880F50
:10281000880F912F9F70C92ED12CE12CF12C082EFE
:1028200004C0CC0CDD1CEE1CFF1C0A94D2F714FF74
:1028300012C04FE050E060E070E004C0440F551F4C
:10284000661F771F8A95D2F7CB01BA016095709504
:102850008095909503C060E070E0CB012B2D26950C
:1028600026952370422F50E042305105D9F0433075
:10287000510569F16C297D298E299F294130510527
:1028800051F126960FB6F894DEBF0FBECDBFDF9193
:10289000CF911F910F91FF90EF90DF90CF90BF905D
:1028A0000C94011A6C297D298E299F2926960FB632
:1028B000F894DEBF0FBECDBFDF91CF911F910F9176
:1028C000FF90EF90DF90CF90BF900C941D1A0E9464
:1028D000011AC701B60126960FB6F894DEBF0FBEE7
:1028E000CDBFDF91CF911F910F91FF90EF90DF90BF
:1028F000CF90BF900C94E519002319F08B2D8170B7
:1029000001C08695882309F478C1812F8295869528
:102910008770880F880F912F9F70C92ED12CE12CC2
:10292000F12C082E04C0CC0CDD1CEE1CFF1C0A94FC
:10293000D2F714FF12C04FE050E060E070E004C036
:10294000440F551F661F771F8A95D2F7CB01BA0136
:10295000609570958095909503C060E070E0CB0124
:102960002B2D269526952370422F50E0423051059D
:10297000D9F04330510569F16C297D298E299F29B1
:102980004130510551F126960FB6F894DEBF0FBEC7
:10299000CDBFDF91CF911F910F91FF90EF90DF900E
:1029A000CF90BF900C94DB1A6C297D298E299F292A
:1029B00026960FB6F894DEBF0FBECDBFDF91CF9144
:1029C0001F910F91FF90EF90DF90CF90BF900C94EC
:1029D000F71A0E94DB1AC701B60126960FB6F894C3
:1029E000DEBF0FBECDBFDF91CF911F910F91FF9042
:1029F000EF90DF90CF90BF900C94BF1A103FD1F1B1
:102A000018F4103E50F4A1C0123F09F463C008F45A
:102A10004CC0133F09F473C098C01F708B2D8F7189
:102A20000023A1F00E94581A812F26960FB6F89421
:102A3000DEBF0FBECDBFDF91CF911F910F91FF90F1
:102A4000EF90DF90CF90BF900C94E8120E94791A1B
:102A5000812F26960FB6F894DEBF0FBECDBFDF9153
:102A6000CF911F910F91FF90EF90DF90CF90BF908B
:102A70000C94EF120023A9F02111BFC08B2D8F7190
:102A800026960FB6F894DEBF0FBECDBFDF91CF9173
:102A90001F910F91FF90EF90DF90CF90BF900C941B
:102AA0009E1A223008F0A9C0E9CF0023A9F08B2D8F
:102AB0008F7126960FB6F894DEBF0FBECDBFDF91A3
:102AC000CF911F910F91FF90EF90DF90CF90BF902B
:102AD0000C94581A002359F38B2D8F7126960FB63C
:102AE000F894DEBF0FBECDBFDF91CF911F910F9144
:102AF000FF90EF90DF90CF90BF900C94791A002355
:102B000099F08B2D8F7126960FB6F894DEBF0FBE0D
:102B1000CDBFDF91CF911F910F91FF90EF90DF908C
:102B2000CF90BF900C94431A26960FB6F894DEBF50
:102B30000FBECDBFDF91CF911F910F91FF90EF900E
:102B4000DF90CF90BF900C94391A0023A9F0222374
:102B500009F4ADCF812F26960FB6F894DEBF0FBED5
:102B6000CDBFDF91CF911F910F91FF90EF90DF903C
:102B7000CF90BF900C94D111222309F4ADCF812FB7
:102B800026960FB6F894DEBF0FBECDBFDF91CF9172
:102B90001F910F91FF90EF90DF90CF90BF900C941A
:102BA00099124B2D4F70612FC7010E943604269653
:102BB0000FB6F894DEBF0FBECDBFDF91CF911F914E
:102BC0000F91FF90EF90DF90CF90BF900C945D1924
:102BD0004B2D4F70612FC70126960FB6F894DEBFBC
:102BE0000FBECDBFDF91CF911F910F91FF90EF905E
:102BF000DF90CF90BF900C944B0826960FB6F894B8
:102C0000DEBF0FBECDBFDF91CF911F910F91FF901F
:102C1000EF90DF90CF90BF9008950E94F81B0E9424
:102C2000CD1B0E94121C0E941D210E946C2080E07E
:102C300090E00E94CB1080E090E00C94E1100E94A4
:102C4000E81B0C940D160E94141B292F22952F703F
:102C500030E02C3031054CF42A3031056CF4225030
:102C600031092230310588F407C02C30310549F094
:102C70002F30310531F009C0803E48F0803F29F403
:102C800006C093FB882780F9089580E0089581E0CD
:102C90000895CF93DF9300D000D01F92CDB7DEB759
:102CA0000F900F900F900F900F90DF91CF9108959C
:102CB000CF93DF9300D000D000D0CDB7DEB72696FB
:102CC0000FB6F894DEBF0FBECDBFDF91CF91089550
:102CD0001F93CF93DF93C0917B0116E080917C011D
:102CE000C81799F0D0E01C9FF0011D9FF00D112432
:102CF000E358FE4F408151816281738184819581C7
:102D00000E9458162196C770E9CFDF91CF911F918D
:102D100008954091AD015091AE016091AF01709165
:102D2000B0018091B1019091B2010C94581680913C
:102D3000B20182958F7009F054C08091AF01882351
:102D400009F44FC080917B01A0917C016091AD019D
:102D50007091AE014091B0015091B101B6E08A1777
:102D600009F43FC090E041155105C1F17F3F11F4D6
:102D70006F3FA1F1B89FF001B99FF00D1124E35806
:102D8000FE4F218172132AC02081621327C0228145
:102D9000211124C0238134812417350710F42150D8
:102DA0003109241B350B283C3105C0F42091B201B8
:102DB0002F7020612093B20126E0289FF001299F07
:102DC000F00D1124EE57FE4F80818F70806180835B
:102DD0008DEA91E00E94F6120C94681601968770B5
:102DE000BECF0895CF92DF92EF92FF920F931F9381
:102DF000CF93DF93CDB7DEB762970FB6F894DEBFFF
:102E00000FBECDBF8C0185E0F801DE011D9601905B
:102E10000D928A95E1F7D8014C9111965C9111972A
:102E200012966C9112971396CD90DC901497309176
:102E3000AD017091AE018091B0019091B101009708
:102E400009F46BC17F3F19F43F3F09F466C1E0907C
:102E5000AF01EE2009F4C0C02091B201C816D90616
:102E600028F0F601E81BF90BCF0104C0809590957E
:102E70008C0D9D1DFF24F394883C910578F0F12C76
:102E8000207F09F0C6C07C2DD98AC88A89890E9412
:102E900049168DEA91E00E94F612B1C0822F807F20
:102EA00009F046C0751314C0341312C0611110C06C
:102EB0002F7020612093B2010E9489168DEA91E063
:102EC0000E94F6128091B201D80115968C932EC003
:102ED000CD2819F15F3F11F44F3FF9F0F62E611143
:102EE0001CC080917B0120917C0136E0821709F49F
:102EF0005AC090E0389FF001399FF00D1124E3583B
:102F0000FE4F7181571306C07081471303C0728151
:102F1000711103C001968770E9CFF62E662309F47C
:102F200018C18091B20181608093B201F12C11C16E
:102F3000751308C0341306C0611104C08091B2013A
:102F4000D801C3C04D875E878D859E856A8B0E94A0
:102F500023166A898823E1F16623D1F12091B20119
:102F6000822F82958F7090E0029774F08091AD016E
:102F70009091AE0198878F831986DB86CA862C874D
:102F8000CE0107960E94F61286E0F801ADEAB1E0A4
:102F900001900D928A95E1F70E9497160E9489167A
:102FA000FF24F394D6C04D875E878D859E850E9451
:102FB000141B292F22952F7030E0223031050CF0A0
:102FC000BCC09F7009F0B6C0805E883008F4C1C0F4
:102FD000C8010E94F612E4CFC816D90608F453C0FF
:102FE000F601E81BF90BCF01883C910508F450C0AD
:102FF000F12C7C2DD98AC88A89890E944916EDEA6C
:10300000F1E086E0DF011D928A95E9F70E948916BA
:10301000A0C0751314C0341312C0611110C0809188
:10302000B201F8018583C8010E94F61286E0EDEA3C
:10303000F1E0DF011D928A95E9F7FE2C8AC04D87E9
:103040005E878D859E856A8B0E9423166A898823F8
:1030500009F4BECF662309F4BBCF2091B201822FC1
:1030600082958F7090E002970CF48ECF8091AD0125
:103070009091AE019A8389831B82DD82CC822E835C
:10308000CE0101967FCF809590958C0D9D1DACCF84
:10309000F62E662309F49CCF75132EC034132CC072
:1030A0002091B20120FD1FC0822F82958F70D9F030
:1030B000D80115962C9315978F3049F08F5F982F74
:1030C0009295907F822F8F70892B15968C93C801D3
:1030D0000E94F61286E0F801ADEAB1E001900D928F
:1030E0008A95E1F793CF86E0F801ADEAB1E001906F
:1030F0000D928A95E1F72DC04D875E878D859E855F
:103100000E942316811140CF8091B201816080938B
:10311000B201C8010E94F6121CC0662309F458CF00
:103120004D875E878D859E850E942316882309F42E
:103130004FCF2ACF811148CF0CC0243031050CF07D
:1031400047CF9F7009F440CFF8019581907F09F037
:103150003BCF8F2D62960FB6F894DEBF0FBECDBF6A
:10316000DF91CF911F910F91FF90EF90DF90CF9063
:1031700008951F93CF93DF93CDB7DEB72C970FB68B
:10318000F894DEBF0FBECDBF4F83588769877A871B
:103190008B879C87CE0107960E94F216882369F0E0
:1031A0008F8198852A853B85232BF1F19F3F09F07C
:1031B00063C08F3F09F060C037C086E0FE013796DC
:1031C000DE01119601900D928A95E1F76F81788565
:1031D000EA85FB85309741F17F3F11F46F3F21F184
:1031E00020917C0130E0C9010196877099274091B8
:1031F0007B0150E08417950709F447C069837A83FF
:10320000FD83EC8396E0929FD001939FB00D112433
:10321000A358BE4FFE01319601900D929A95E1F7A9
:1032200080937C010E94681616E080917B0190914A
:103230007C018917C1F1189FC001112483589E4F4A
:103240000E94F216882379F1E0917B011E9FF00124
:103250001124E358FE4F4081518162817381848142
:1032600095810E94581680917B0190E001968770AD
:10327000992780937B01D9CF4F81588569857A85BD
:103280008B859C850E945816CFCF0E941F161092E6
:103290007C0110927B01EDEAF1E086E0DF011D92F6
:1032A0008A95E9F7C1CF2C960FB6F894DEBF0FBE12
:1032B000CDBFDF91CF911F910895EF92FF920F93B1
:1032C0001F93CF93DF938C01892B09F46CC0F12CF1
:1032D000EE24E394E8012196F8018491843740F4C8
:1032E000843008F051C0813081F0823019F15BC028
:1032F000853709F444C0A8F19CE7980F903708F08F
:1033000052C08F770E94991241C00E5F1F4FFE017D
:10331000C49180E28C0F883048F4C7708E2D01C0B4
:10332000880FCA95EAF70E94EB1B14C08C2F0E94ED
:10333000D1112DC00E5F1F4FFE01C49180E28C0F92
:10334000883058F4C7708E2D01C0880FCA95EAF7EF
:103350000E94F11B0E94121C1AC08C2F0E9499120D
:1033600016C00E5F1F4FFE01C491CC2381F08FE980
:103370009FE00197F1F700C00000C150F6CF0E5F4B
:103380001F4FFE01F49003C00E94D1118E018F2DBA
:10339000882309F49FCFEFE9FFE03197F1F700C0F0
:1033A00000008150F5CFDF91CF911F910F91FF90D9
:1033B000EF90089508956093B7017093B8018093DA
:1033C000B9019093BA010C940D160F931F930091BD
:1033D000B7011091B8012091B9013091BA01DC0117
:1033E000CB01802B912BA22BB32B8093B701909311
:1033F000B801A093B901B093BA011F910F910C9439
:103400000D160F931F930091B7011091B8012091F1
:10341000B9013091BA01DC01CB0180239123A223B1
:10342000B3238093B7019093B801A093B901B093EF
:10343000BA011F910F910C940D160F931F930091D9
:10344000B7011091B8012091B9013091BA01DC01A6
:10345000CB0180279127A227B3278093B7019093B0
:10346000B801A093B901B093BA011F910F910C94C8
:103470000D161092B3011092B4011092B501109282
:10348000B6010C940D1641E050E060E070E004C01D
:10349000440F551F661F771F8A95D2F74093B301DB
:1034A0005093B4016093B5017093B6010C940D165E
:1034B00041E050E060E070E004C0440F551F661F1B
:1034C000771F8A95D2F78091B3019091B401A091B2
:1034D000B501B091B601482B592B6A2B7B2B409339
:1034E000B3015093B4016093B5017093B6010C948D
:1034F0000D1641E050E060E070E004C0440F551F3D
:10350000661F771F8A95D2F7409550956095709504
:103510008091B3019091B401A091B501B091B60131
:10352000482359236A237B234093B3015093B4016A
:103530006093B5017093B6010C940D1641E050E014
:1035400060E070E004C0440F551F661F771F8A9526
:10355000D2F78091B3019091B401A091B501B091DF
:10356000B601482759276A277B274093B301509318
:10357000B4016093B5017093B6010C940D160F93CE
:103580001F930091B3011091B4012091B5013091C6
:10359000B601DC01CB01802B912BA22BB32B8093A6
:1035A000B3019093B401A093B501B093B6011F91FC
:1035B0000F910C940D160F931F930091B30110916E
:1035C000B4012091B5013091B601DC01CB0180231B
:1035D0009123A223B3238093B3019093B401A093CA
:1035E000B501B093B6011F910F910C940D160F9376
:1035F0001F930091B3011091B4012091B501309156
:10360000B601DC01CB0180279127A227B327809345
:10361000B3019093B401A093B501B093B6011F918B
:103620000F910C940D160895CF92DF92EF92FF92B6
:103630000F931F93CF93DF938C01C090B701D0906D
:10364000B801E090B901F090BA014091B3015091F6
:10365000B4016091B5017091B601C42AD52AE62A59
:10366000F72ACFE1D0E0D701C6010C2E04C0B695F1
:10367000A795979587950A94D2F780FF07C0B80160
:103680008C2F0E946E088130910531F4219758F7F4
:10369000B80180E00E946E08DF91CF911F910F91D9
:1036A000FF90EF90DF90CF90089590910C019923B7
:1036B00021F090910D01911109C020910E013091DE
:1036C0000F01F90132969FEF40E01FC0982F9695A9
:1036D000969596959F3050F5E0910E01F0910F016F
:1036E000E90FF11D877021E030E0A90102C0440F0D
:1036F000551F8A95E2F7CA019181892B818308952C
:103700009F3F39F04F5F4E3041F051915813F8CF41
:103710000DC05111F7CF942FF5CF9F3F39F0F9012C
:10372000E90FF11D97FDFA95828308950895909110
:103730000C01992321F090910D01911109C0209164
:103740000E0130910F01F9013296205F3F4F1FC0EB
:10375000982F9695969596959F30F0F4E0910E01EE
:10376000F0910F01E90FF11D877021E030E0A90110
:1037700002C0440F551F8A95E2F7CA0180959181D6
:103780008923818308953196E217F30729F0908108
:103790009813F9CF1082F7CF089581E090E0E0917F
:1037A0000E01F0910F01E80FF91F10820196803190
:1037B0009105A9F708959091CD01892B8093CD01B2
:1037C000089580959091CD0189238093CD0108952E
:1037D0001092CD0108959091CC01892B8093CC015A
:1037E000089580959091CC0189238093CC01089510
:1037F0001092CC0108958093BB0108951092BB01F3
:10380000089580910E0190910F01FC0131969C0169
:10381000205F3F4F80E0919191118F5FE217F30796
:10382000D1F70895E0910E01F0910F018091CD0143
:103830008083E0910E01F0910F0190818091CC0185
:10384000892B80838091BB01882361F0E0910E0178
:10385000F0910F019081892B80830E94011C8111BE
:103860001092BB0180910E0190910F010C94B51044
:10387000CF92DF92EF92FF926C01EE24FF24C114ED
:10388000D104E104F10421F0C701B60120E101C037
:1038900020E0C72ED82EE92EFF24C114D104E10464
:1038A000F10419F0285FC701B6016B017C0154E0F7
:1038B000F694E794D794C7945A95D1F7C114D104DC
:1038C000E104F10419F02C5FC701B6016B017C0122
:1038D00042E0F694E794D794C7944A95D1F7C1147F
:1038E000D104E104F10419F02E5FC701B601DC0137
:1038F000CB01B695A79597958795892B8A2B8B2B0E
:1039000009F02F5F822FFF90EF90DF90CF90089506
:103910008091E701843009F11092CF0120E488E121
:1039200090E00FB6F894A895809360000FBE2093A6
:10393000600083B7817F846083BF83B7816083BF6A
:103940007894889583B78E7F83BF88E10FB6F8940B
:1039500080936000109260000FBE0895089508954E
:10396000CF930E94AE1C0E9497060E94AF1CC0E03D
:103970008C2F0E948507811104C0CF5FCE30C1F724
:1039800001C081E0CF9108950E941F160E94A910E6
:103990000C94A20982E084BD93E095BD9AEF97BD97
:1039A00080936E0008952FB7F8948091D001909184
:1039B000D101A091D201B091D3012FBF0895CF9230
:1039C000DF92EF92FF920F931F932FB7F8944091DD
:1039D000D0015091D1016091D2017091D3012FBFDC
:1039E0006A017B01EE24FF248C0120E030E0C01648
:1039F000D106E206F30610F4415051099A01281B42
:103A0000390BC9011F910F91FF90EF90DF90CF907C
:103A100008951F920F920FB60F9211248F939F93C8
:103A2000AF93BF938091D0019091D101A091D20129
:103A3000B091D3010196A11DB11D8093D001909347
:103A4000D101A093D201B093D301BF91AF919F91C7
:103A50008F910F900FBE0F901F9018950E94A60D8A
:103A6000F8942FEF87EA91E6215080409040E1F7EB
:103A700000C0000087E090EBDC018093F0019093A0
:103A8000F101A093F201B093F3019CE088E10FB63D
:103A9000F894A895809360000FBE90936000FFCFCC
:103AA000EF92FF920F931F93CF93DF93D82FC0E035
:103AB0008C2F0E94850700E010E0E82EF12CC70152
:103AC000002E02C0959587950A94E2F780FD06C006
:103AD0000F5F1F4F0630110591F709C0602F7C2F33
:103AE00080E00E944C08D813F3CF81E004C0CF5F80
:103AF000CE30F1F680E0DF91CF911F910F91FF90D2
:103B0000EF900895CF93C82F8CE20E94501D882318
:103B100021F08C2FCF910C94501D80E0CF9108950F
:103B2000CF930E94D71E811102C00E94BD1EC5E620
:103B3000C15049F00E9497068FE39CE90197F1F785
:103B400000C00000F5CF89E20E94821D811113C1DF
:103B50008AE20E94821D81110E94BD1E85E00E94A2
:103B6000821D81110E942E1D0E94E21E8093CE01B3
:103B700087E00E94821D8823A9F18BE10E94821DAB
:103B8000882351F08091CE0181FB222720F991E01A
:103B9000922790FB81F90EC08EE00E94821D88233F
:103BA00061F08091CE0182FB222720F991E09227DB
:103BB00090FB82F98093CE0115C080E10E94821DA6
:103BC0009091CE01882341F093FB222720F981E0D8
:103BD000822780FB93F904C0892F809580FB90F9A0
:103BE0009093CE018091CE010E94E61E0E94F41EA9
:103BF0008093E10180EE0E94821D882341F0809134
:103C0000E101982F909590FB80F98093E10189E381
:103C10000E94821D882359F08091E10181FB2227B7
:103C200020F991E0922790FB81F98093E10182EEE7
:103C30000E94821D882359F08091E10182FB222796
:103C400020F991E0922790FB82F98093E10186EEC2
:103C50000E94821D882359F08091E10183FB222775
:103C600020F991E0922790FB83F98093E10183EEA4
:103C70000E94821D882359F08091E10184FB222754
:103C800020F991E0922790FB84F98093E10185E38C
:103C90000E94821D882359F08091E10185FB222733
:103CA00020F991E0922790FB85F98093E10181E36F
:103CB0000E94821D882359F08091E10186FB222712
:103CC00020F991E0922790FB86F98093E10181E150
:103CD0000E94821D882359F08091E10187FB2227F1
:103CE00020F991E0922790FB87F98093E101809180
:103CF000E1010E94F81E8091E10187FB882780F98D
:103D000080930D0187E20E94821DC82F8EE10E94E0
:103D1000821D8111C2608FE10E94821D8111C460E9
:103D200080E20E94821D8111C86081E20E94821D92
:103D30008111C06182E20E94821D8111C06283E212
:103D40000E94821D8111C06484E20E94821D88232A
:103D500011F0C06802C0CC2329F08C2F0E94EF1E06
:103D60006C2F03C00E94EB1E682F70E080E090E093
:103D7000CF910C94DB19CF9108956DEE7EEF80E02A
:103D800090E00E94232560E082E090E00E941525EB
:103D900060E083E090E00E94152560E084E090E020
:103DA0000E94152560E085E090E00C94152580E0E8
:103DB00090E00E940F2521E08D3E9E4F09F020E00B
:103DC000822F089582E090E00C940725682F82E00E
:103DD00090E00C94152583E090E00C940725682F63
:103DE00083E090E00C94152584E090E00C94072586
:103DF000682F84E090E00C9415258091D60180FF17
:103E00000BC06091130185E0689FB0011124759586
:103E10006795759567952BC081FF09C06091130167
:103E200085E0689FB00111247595679520C082FFD9
:103E300007C06091130185E0689FB001112417C08D
:103E40009091D7019923D1F060911201961788F7CC
:103E50002091130185E0289F90011124929FA001D9
:103E6000939F500D112470E0CA010E94D92460383C
:103E7000710540F46115710539F002C065E070E02C
:103E8000862F08958FE7089581E008958091D601E7
:103E900080FF08C06091110170E075956795759578
:103EA000679521C081FF06C06091110170E0759592
:103EB000679519C082FF04C06091110170E010C0C5
:103EC0009091D7019923C1F0609110019617A0F746
:103ED00080911101899FC001112470E00E94D924B2
:103EE0006038710528F46115710521F0862F089559
:103EF0008FE7089581E0089561E070E0F4CF803F9E
:103F000021F40E94FD1E819504C0813F29F40E9486
:103F1000FD1E8093DA010895823F21F40E94FD1E68
:103F2000819504C0833F29F40E94FD1E8093D9012E
:103F30000895893F19F40E94461F05C08A3F31F455
:103F40000E94461F81958093DB0108958B3F21F4E9
:103F50000E94461F819504C08C3F29F40E94461F91
:103F60008093DC010895843F21F48091D801816021
:103F700017C0853F21F48091D801826011C0863F2F
:103F800021F48091D80184600BC0873F21F4809197
:103F9000D801886005C0883F31F48091D8018061E4
:103FA0008093D80108958D3F21F48091D6018160DE
:103FB0000BC08E3F21F48091D601826005C08F3FF7
:103FC00029F48091D60184608093D6010895803FC2
:103FD00039F48091DA0187FF6CC01092DA0169C070
:103FE000813F29F48091DA011816BCF362C09091E8
:103FF000D901823F29F497FF5CC01092D90159C0C2
:10400000833F19F41916CCF354C0893F41F48091D1
:10401000DB0118160CF04DC01092DB014AC08A3F3C
:1040200029F48091DB0187FF44C0F6CF8B3F39F440
:104030008091DC0187FF3DC01092DC013AC08C3FCB
:1040400029F48091DC011816BCF333C0843F21F4BD
:104050008091D8018E7F17C0853F21F48091D801CF
:104060008D7F11C0863F21F48091D8018B7F0BC0DA
:10407000873F21F48091D801877F05C0883F31F4C4
:104080008091D8018F7E8093D80113C08D3F21F499
:104090008091D6018E7F0BC08E3F21F48091D60196
:1040A0008D7F05C08F3F29F48091D6018B7F80934F
:1040B000D6018091D90181110EC08091DA01811160
:1040C0000AC08091DB01811106C08091DC01811161
:1040D00002C01092D701089588ED91E00E94C010AF
:1040E0000E94D31C9093D5018093D40108951F930F
:1040F000CF93DF938091D4019091D5010E94DF1C72
:10410000AC019091D701992321F02091140130E066
:1041100006C0209115018AE0289F900111244217C2
:10412000530708F486C08091D901C091DA01D0917B
:10413000DB011091DC01811107C0C11176C0D111E2
:1041400074C0111172C075C09F3F19F09F5F9093AA
:10415000D701181624F40E94FD1E8093D901809186
:10416000D90187FF05C00E94FD1E81958093D9016A
:104170001C1624F40E94FD1E8093DA018091DA015E
:1041800087FF05C00E94FD1E81958093DA01609132
:10419000D901662339F1C091DA01CC2319F17727CF
:1041A00067FD7095872F972F0E94EA2323E333E35F
:1041B00043E35FE30E944E240E94B7236093D9013A
:1041C0006C2F772767FD7095872F972F0E94EA2322
:1041D00023E333E343E35FE30E944E240E94B723CB
:1041E0006093DA011D1624F40E94461F8093DB01C0
:1041F0008091DB0187FF05C00E94461F8195809357
:10420000DB01111624F40E94461F8093DC0180918B
:10421000DC0187FF05C00E94461F81958093DC0169
:10422000DF91CF911F910C946C209F3F09F08ECFAE
:1042300096CFDF91CF911F910895E8EDF1E085E0F1
:10424000DF011D928A95E9F71092D7011092D601ED
:104250000895833081F128F4813059F08230D1F013
:104260000895853009F449C0B8F1863009F456C084
:10427000089580911501262F30E0280F311D2F3F22
:10428000310524F4680F6093150108958FEF809332
:104290001501089580911401262F30E0280F311D5B
:1042A0002F3F310524F4680F6093140108958FEFB8
:1042B00080931401089580911301262F30E0280F78
:1042C000311D2F3F310524F4680F609313010895C9
:1042D0008FEF80931301089580911201262F30E013
:1042E000280F311D2F3F310524F4680F6093120110
:1042F00008958FEF80931201089580911101262F68
:1043000030E0280F311D2F3F310524F4680F6093F2
:10431000110108958FEF809311010895809110018C
:10432000262F30E0280F311D2F3F310524F4680F70
:104330006093100108958FEF8093100108958330EA
:1043400011F128F4813049F0823091F008958530E0
:1043500081F120F18630C1F108958091150168172F
:1043600020F4861B8093150108951092150108957D
:1043700080911401681720F4861B8093140108951E
:1043800010921401089580911301681720F4861B80
:1043900080931301089510921301089580911201E2
:1043A000681720F4861B8093120108951092120161
:1043B000089580911101681720F4861B80931101E4
:1043C000089510921101089580911001681720F44A
:1043D000861B8093100108951092100108950F9389
:1043E0001F938D3109F46BC008F03FC08E3009F483
:1043F0007DC0C0F4873009F46EC068F4863009F0DF
:10440000AFC08091CE01817F8E7F8093CE0181E00D
:104410008093DE01A6C0883009F458C08B3009F4BF
:104420009BC09EC0863109F497C078F4803109F4AE
:1044300070C0813109F094C00E941F1690910D0147
:1044400081E0892780930D0187C0893109F484C0F8
:104450008B3109F085C08091CE0181FB222720F9A4
:1044600091E0922790FB81F94AC0853309F45BC043
:1044700048F4873209F457C008F45AC0893209F465
:1044800052C06EC0833438F48A3308F067C0883372
:1044900009F462C065C0833409F445C0883409F06A
:1044A0005FC00E941F160FEF13ED20E30150104074
:1044B0002040E1F700C000000E942E1D4DC00E9468
:1044C00071230E94A9100E94A20946C00E94E21E08
:1044D0000E94F41E41C09091CE01892F817090FFFF
:1044E00012C0917F9E7F9093CE013BC08091CE0100
:1044F00082FB222720F991E0922790FB82F980939A
:10450000CE01992349F18091CE0181608093CE0143
:1045100023C08091CE0183FB222720F991E09227CE
:1045200090FB83F9ECCF61E070E080E090E010C098
:104530008D5141E050E060E070E08A019B0104C0D1
:10454000000F111F221F331F8A95D2F7C901B8012E
:104550000E94DB190E941F1681E003C08953E9CF36
:1045600080E01F910F91089580E0089580E0089504
:10457000CF93C82F8091DE01813079F018F082301E
:10458000E9F187C0E0910E01F0910F018081813146
:1045900069F0823209F07FC009C0E0910E01F0910C
:1045A0000F018081813111F0823261F48C2F0E94E1
:1045B000B422811104C08C2F0E94EF211DC081E024
:1045C00090E01AC08C2F0E94B622811114C0C43111
:1045D00079F048F4CB3079F0C03109F060C082E066
:1045E0008093DE0108C0C93219F0C83321F057C0EA
:1045F0001092DE0154C081E0817053C0C93289F14C
:1046000018F5C43171F1A8F4C73009F046C08AE04A
:104610008093150194E19093140193E0909313011A
:104620008093120188E08093110188E28093100149
:1046300034C0CE51C63088F5EC2FF0E0E65DFE4F79
:1046400080818093DD0129C0CE34E9F020F4CB34A1
:1046500021F56AE013C0C13579F0C235F1F461E0AB
:104660000DC08091DD01882319F01092DD0115C085
:1046700081E08093DE0115C061E006C08091DD011C
:104680000E9429210AC06AE08091DD010E949F21D9
:1046900004C01092DE0180E004C081E002C080E02E
:1046A000ABCFCF910895E1E8F0E08081886080830E
:1046B0008081816080838FB7F89493E09093890024
:1046C00090ED909388008FBF0895EFE6F0E0808131
:1046D000826080830895EFE6F0E080818D7F8083A3
:1046E0000895EFE6F0E0908182E0892780830895C5
:1046F0001F920F920FB60F9211242F933F934F9357
:104700005F936F937F938F939F93AF93BF93EF9339
:10471000FF938091DF019091E00101969093E00179
:104720008093DF01811103C082E00E94A209E09121
:10473000E001E695E695F0E0E156F84FE4918091CE
:10474000DF018E1303C080E00E94A209FF91EF9168
:10475000BF91AF919F918F917F916F915F914F9199
:104760003F912F910F900FBE0F901F90189504D07E
:104770006894B1118DC0089570D088F09F5790F063
:10478000B92F9927B751A0F0D1F0660F771F881F76
:10479000991F1AF0BA95C9F712C0B13081F077D0DD
:1047A000B1E0089574C0672F782F8827B85F39F07B
:1047B000B93FCCF3869577956795B395D9F73EF4D5
:1047C00090958095709561957F4F8F4F9F4F08957D
:1047D000E89409C097FB3EF490958095709561959B
:1047E0007F4F8F4F9F4F9923A9F0F92F96E9BB2751
:1047F0009395F695879577956795B795F111F8CFCD
:10480000FAF4BB0F11F460FF1BC06F5F7F4F8F4F37
:104810009F4F16C0882311F096E911C0772321F02D
:104820009EE8872F762F05C0662371F096E8862FC5
:1048300070E060E02AF09A95660F771F881FDAF71C
:10484000880F9695879597F9089557FD9058440FCE
:10485000551F59F05F3F71F04795880F97FB991FDF
:1048600061F09F3F79F0879508951216130614069C
:10487000551FF2CF4695F1DF08C016161706180629
:10488000991FF1CF86957105610508940895E89404
:10489000BB2766277727CB0197F908950BD078C0FF
:1048A00069D028F06ED018F0952309F05AC05FC087
:1048B0001124EECFCADFA0F3959FD1F3950F50E0FE
:1048C000551F629FF001729FBB27F00DB11D639FC2
:1048D000AA27F00DB11DAA1F649F6627B00DA11D68
:1048E000661F829F2227B00DA11D621F739FB00D0E
:1048F000A11D621F839FA00D611D221F749F33277E
:10490000A00D611D231F849F600D211D822F762F16
:104910006A2F11249F5750408AF0E1F088234AF013
:10492000EE0FFF1FBB1F661F771F881F915050405F
:10493000A9F79E3F510570F014C0AACF5F3FECF37A
:10494000983EDCF3869577956795B795F795E7954B
:104950009F5FC1F7FE2B880F911D9695879597F95C
:10496000089597F99F6780E870E060E008959FEFF1
:1049700080EC089500240A941616170618060906F6
:10498000089500240A9412161306140605060895C5
:10499000092E0394000C11F4882352F0BB0F40F44D
:1049A000BF2B11F460FF04C06F5F7F4F8F4F9F4F8D
:1049B000089597FB072E16F4009407D077FD09D0D1
:1049C0000E94F32407FC05D03EF4909581959F4FFB
:1049D0000895709561957F4F0895EE0FFF1F059024
:1049E000F491E02D0994AA1BBB1B51E107C0AA1F3B
:1049F000BB1FA617B70710F0A61BB70B881F991F80
:104A00005A95A9F780959095BC01CD010895F99923
:104A1000FECF92BD81BDF89A992780B50895A8E18F
:104A2000B0E042E050E00C942A25262FF999FECF01
:104A30001FBA92BD81BD20BD0FB6F894FA9AF99ABB
:104A40000FBE019608950E941525272F0C94162558
:104A5000DC01CB01FC01F999FECF06C0F2BDE1BD3E
:104A6000F89A319600B40D9241505040B8F708952D
:044A7000F894FFCFE8
:104A74002002A409320A0F0ADB09A7090101BC01BB
:104A840028080A03140A3F4D363960071307DD0668
:104A9400A4063706500669068206010203040506C9
:044AA40007080900F6
:00000001FF
